:100000000200081200B580FE7581091200EEE5823B
:1000100060030200037900E94400601B7A0090004D
:10002000F2780075A000E493F2A308B8000205A0DE
:10003000D9F4DAF275A0FFE478FFF6D8FD7800E88D
:100040004400600A790075A000E4F309D8FC780048
:10005000E84400600C7900900000E4F0A3D8FCD9DB
:10006000FA020003AA82AB83EA4B700490000122DB
:10007000BA0107BB000490000122EA24FFF582EBDD
:1000800034FFF583C002C0031200648582088583B3
:1000900009D003D0028A828B830200D14398404367
:1000A0008920758DFD43878022AA82AB83C2998AFD
:1000B000993099FD2212009C90000A1200A990002C
:1000C000141200A99000031200641200A990000508
:1000D00022E5828508F0A4C582C0F08509F0A4D08D
:1000E000F025F0C5838508F0A42583F58322758269
:0200F0000022EC
:00000001FF
